:10000000F01F0010253500002135000021350000CB
:1000100021350000213500002135000000000000DE
:10002000000000000000000000000000213500007A
:1000300021350000000000002135000051130000B0
:10004000FD100000FD100000FD100000FD1000007C
:10005000FD100000FD100000FD100000FD1000006C
:10006000FD100000FD100000FD100000FD1000005C
:10007000FD1000001D3500001D3500001D3500007D
:10008000091400002114000039140000511400006C
:100090001D350000311500001D3500001D35000024
:1000A0001D3500001D3500001D3500001D35000008
:1000B0001D3500001D3500001D3500001D350000F8
:1000C00008B500230B60036000F096FD08BD08B57D
:1000D0000A20002101F038F908BD000038B50C4BAA
:1000E0000D1C041C19680B4803F050FA212103F081
:1000F0004DFA011C012001F0D7F9012001F0B4F9FB
:10010000291C201C02F084FD012001F0BDF938BD3E
:1001100078800440001BB70008B50A4B0A481968EC
:1001200003F034FA212103F031FA011C012001F01F
:10013000BBF9012001F098F902F0ECFC012001F07C
:10014000A3F908BD78800440001BB70013B59620C2
:10015000000201F02BFA18480D210C2200F02CFCB3
:1001600000F06AFB15480021032200F099FC00F022
:100170006DFBFFF7D1FF1248124901F0FFFB00248D
:1001800001F0BEFA002802D000F0E0FE00240A20B0
:1001900001F00AF9684601A9FFF792FF009B002BC6
:1001A00003D1094B01349C42EADDFFF7B5FF074854
:1001B00001F0E4FB13BDC0464E3900005437000087
:1001C000633700006E3700006F17000075370000BE
:1001D00007B5044B04490093044A054B01F0D9FBD1
:1001E00007BDC04691370000803700006E37000021
:1001F0008937000070B50D1C161C041C00F01CFB98
:100200000B480D210C2200F0D7FB281CA1B20022C4
:1002100000F046FC07480321062200F0CDFB301C0D
:100220000121092200F03CFC00F010FB70BDC0462B
:100230004E3900000938000038B50D1C041C00F0D0
:10024000DAFA2A1C0120211CFFF7D4FF034B0022FD
:100250005A60034A943212689A6038BD281300101D
:100260008C04001010B588B0041C6846FFF7B0FF7E
:1002700069466A46201CFFF7BDFF08B010BD0000AC
:1002800073B518200021FFF729FF00243B4E012001
:1002900001F0FAF83A4D9835002C01D0002000E02A
:1002A0000620012101F050F8684601A9FFF708FF78
:1002B000009B002B21D1002CF0D12B68002B0DD0FE
:1002C000304B00941A6811321A6004E002F0CCFB43
:1002D000009B01330093009B102BF7DD2A4BF6188F
:1002E000DED518200021FFF7F9FE254B94331C685A
:1002F00063425C4100F074FACEE7002C03D0182B67
:10030000C5D100F0ABFA009B182B1BD1019BC22B6F
:1003100008D11E4B1A6801321A60022A0BD1002242
:100320001A6008E0832B06D10020FFF79BFFFFF740
:10033000F3FEFFF7CCFE019B732B01D1FFF706FF05
:1003400000230193124B1348196803F01FF9212170
:1003500003F01CF9011C012001F0A6F8012001F0B6
:1003600083F80098019902F053FC054B94331B6805
:10037000002B8AD100F034FA012487E720BF020065
:100380008C040010C00200100CFEFFFF7001001072
:1003900078800440001BB70013B501F069FB00F042
:1003A000F7FB00F05BFA00F0DDFD3C24201CFFF7BA
:1003B00059FF013C1E2000F0F7FF022CF6D102F09D
:1003C00075FA1E2300930B2301930E480E4B0F4921
:1003D0000F4A02F025FB00200421012200F0DEFD7F
:1003E0000020021C042100F027FE0020052101222C
:1003F00000F0D4FD00200521021C00F01DFEFFF7D7
:100400003FFFC046E9340000C0020010C1000000F8
:100410003902000000B500E001300378202BFBD04A
:1004200000BD00B5031C303BDAB2092A01D8181C04
:1004300008E020231843031C613B5738052B01D9E2
:100440000120404200BD70B50E1CFFF7E3FF002500
:10045000041C06E0FFF7E5FF002805DB2D0105433E
:10046000013420780028F5D13560201C70BD0000D3
:1004700070B5054E051C0E24013C295D301C01F0B1
:100480007DFA002CF8D170BD9437000000B50E2322
:10049000013BC25C002A03D1002BF9D1012000E00E
:1004A000002000BDF8B500240E2703231C4221D1F3
:1004B0003E1C66432B4D7019FFF7E8FF002815D04E
:1004C000601C78434019FFF7E1FF00280ED0301C74
:1004D0001C304019FFF7DAFF002807D02A367019C0
:1004E000FFF7D4FF002801D004340DE01E48211C82
:1004F00001F044FA381C60431A4B0134C018FFF76E
:10050000B7FF1A4801F03AFAFF2CCEDD184801F087
:1005100035FA184C201CFFF7ABFF174D4221281C61
:1005200001F02CFA201C0E30FFF7A2FF4321281CFB
:1005300001F024FA201C1C30FFF79AFF0F4801F04D
:100540001DFA201C2A30FFF793FF281C4E2101F0D2
:1005500015FA201C3830FFF78BFF616D084801F059
:100560000DFAF8BD2805001097370000315D000036
:10057000A03700008C040010A6370000AD37000043
:10058000B337000070B50E1CFFF744FF0D25041CA7
:100590002078FFF746FF002807DB01347055013D46
:1005A000F6D2201CFFF736FF00E0002070BD0000EF
:1005B00073B5394D08682B78002B06D1374801F008
:1005C000DDF902F073F9012342E00378412B1BD1DE
:1005D000334C0230211CFFF7D5FF002851D003789F
:1005E000422B4ED1211C02300E31FFF7CBFF0028E9
:1005F00047D00378432B44D1211C02301C31FFF734
:10060000C1FF002846D13CE04D2B23D1254C0230C0
:10061000211CFFF7B7FF002833D003784E2B30D1D1
:10062000211C02300E31FFF7ADFF002829D00378DE
:10063000472B26D1023001A9FFF705FF019B002BB4
:100640001FDB2A3C63651848184901F097F900231D
:100650002B701FE001A9FFF7F6FE0378202B01D0D5
:10066000002B0ED1124E00240E250199611869430A
:100670008919FFF787FF002803D00134042CF4D137
:1006800008E002F013F908480A4901F077F9024B33
:1006900000221A7073BDC04698020010BF370000D8
:1006A0008C040010B6040010D5370000DF370000BE
:1006B00028050010E237000037B54C6824E0201C04
:1006C000FFF7A8FE01A9FFF7BEFE019B041C002B4B
:1006D0001DD0D8B2FF2B09DD00F0FCF9051C0198F4
:1006E0000012C0B200F0F6F9019003E000F0F2F958
:1006F000002501900198002802D0291CFFF7EEFC8C
:1007000023785A1E9341E4182378002BD7D137BDA4
:1007100008B5064A012113784B40137001D00449F3
:1007200000E00449044801F029F908BD79030010EC
:10073000E9370000F1370000FA37000070B5051CFA
:1007400001200821021C00F077FC0724012601206B
:100750000821002200F070FC2A1C224132400020B7
:10076000022100F069FC01200821021C00F064FC59
:10077000013CECD270BD10B50021041C0A1C022003
:1007800000F05AFC201CFFF7D9FF10BDF7B501237C
:1007900000930023019372B66C46061C02AF01CC95
:1007A00050235B421843C0B2FFF7E5FF0020FFF77C
:1007B000E2FF1020FFF7DFFFE020FFF7DCFF00255E
:1007C00002200021012200F037FC705D0135FFF7A7
:1007D000B5FF842DF4D18436BC42E0D162B6F7BDBA
:1007E00008B5AC20FFF7C7FFAE20FFF7C4FFA52078
:1007F000FFF7C1FF08BD08B5AF20FFF7BCFFA4207D
:10080000FFF7B9FF08BD08B5AE20FFF7B4FF08BD7C
:1008100010B5041CF820FFF7AEFF201CFFF7ABFF5C
:1008200010BD10B5041C8120FFF7A5FF3F2020401C
:10083000FFF7A1FF10BD000008B584220248002187
:10084000520001F0D3F808BD8103001008B502483A
:10085000FFF79CFF08BDC0468103001008B50120CA
:10086000021C082100F09AFB0120021C082100F064
:10087000E3FB00200221012200F090FB0020022176
:10088000012200F0D9FB02200021012200F086FBAA
:1008900002200021012200F0CFFB022006210122CC
:1008A00000F07CFB02200621012200F0C5FB0320A2
:1008B000011C012200F072FB0320011C012200F048
:1008C000BBFB0320011C002200F0B6FB0220062126
:1008D000002200F0B1FB06210122022000F0ACFB57
:1008E000FFF7AAFFFFF7B2FFA220FFF744FFA02007
:1008F000FFF741FFC020FFF73EFF0020FFF788FF12
:100900000A2000F051FD4020FFF735FF2C20FFF7B3
:1009100032FF322000F048FD2E20FFF72CFF32205E
:1009200000F042FD2F20FFF726FF0A2000F03CFDDB
:100930002520FFF720FFAF20FFF71DFFA420FFF7C2
:100940001AFF0020FFF76DFF08BD000000B50F295A
:100950000ED883280CD8CB08842253430722C01812
:100960001140044B80220A41111C1A5C1143195496
:1009700000BDC04681030010F0B55B18DBB216E085
:100980008425CC086C4307270F40802504193D417E
:10099000EFB2A6189C4605E0064BE5182B7801340B
:1009A0003B432B70B442F7DB01316346C9B2994235
:1009B000E6D3F0BD8103001000B5084B1860084B6A
:1009C0001970084B20211A70074B1970074BD1087A
:1009D0001970500701D00131197000BD7C0300105F
:1009E000890400108B0400108A040010800300109A
:1009F000F0B5284B89B01B780024C01A264B06920C
:100A000005911B68221C04E002310C190132A4B2CA
:100A1000D2B2195D8242F7DB1B195B780391029316
:100A200000222CE000994B4303999A198A4214DA68
:100A3000194A0025126892191219D3189B78049349
:100A40000123049AAB40134204D07919C9B2079824
:100A5000FFF77CFF0135082DF2D101360837F6B2D9
:100A6000FFB206E00099059A069F8B18DBB20026BC
:100A700007930A490B789E42D4D3019A013201921E
:100A80006B461B79029900938B42EBD309B0081C8B
:100A9000F0BDC0468A0400107C03001080030010E3
:100AA000F7B5171C061C0D1C00F0C0FF80B20190AA
:100AB0000024FFB208E0305DE9B23A1CFFF798FF6E
:100AC00001302D18ADB20134019AA3B29342F2D392
:100AD000F7BD000000B50F23020918408000031F76
:100AE00000D52833002B0EDB511E032088428041A5
:100AF0004042002807D1242B06DC04218A1A03492E
:100B0000CB18985C00E0002000BDC046513D0000BD
:100B100010B5041C211C144800F0B2FA211C134823
:100B200000F0AEFA211C124800F0AAFA211C11486C
:100B300000F0A6FA211C104800F0A2FA211C0F4870
:100B400000F09EFA211C0E4800F09AFA211C0D4874
:100B500000F096FA211C0C4800F092FA0B48211C78
:100B600000F08EFA10BDC0462040044024400440EE
:100B7000284004402C400440384004403C4004409D
:100B80004040044044400440484004404C4004403D
:100B9000F8B51020FFF7BCFF094C271C1437257847
:100BA0006678281C311C002200F0F8F90234281C59
:100BB000311C012200F040FABC42F0D1F8BDC04621
:100BC000793D0000F8B50B4C271C14372578667862
:100BD000281C311C012200F0E1F90234281C311CD0
:100BE000002200F029FABC42F0D10020FFF790FF6C
:100BF000F8BDC046793D0000F0B589B000240490EE
:100C00000591FFF7C5FF02200721012206940794F2
:100C100000F0C4F902200721221C00F00DFA201C6C
:100C20000B2100F0DFF9A04202D118230693012422
:100C30000021264D03916A782F78111C0192381CEF
:100C4000012200F0ABF9381C0199002200F0F4F900
:100C500003231F4E029314E03078717800F0C2F93C
:100C6000002807D103991B4AA3008A5C1833694600
:100C70005A500134029A039B013A013302920393C2
:100C8000023EE30F00210122A2424B41DBB28B4224
:100C900002D0029B8B42DFDA381C0199002200F05F
:100CA0007DF90199381C012200F0C6F90A49023584
:100CB0008D42C0D1201E06D0069B049A0599136070
:100CC000079B01200B6009B0F0BDC046793D0000D4
:100CD0004F3D0000513D00008D3D000000B50A4B26
:100CE00000211960094B01221A6019601A60196805
:100CF0001142FCD0064B01221A60064B8022196873
:100D000052020A431A6000BD70800440748004409F
:100D1000788004408080044008B500F031F90C4B25
:100D200003201A68120B12031A600A4B1A68120B7E
:100D300012031A60084B1A68120B12031A60074B51
:100D40001A68120B12031A60FFF7C8FF08BDC046ED
:100D5000008000500080015000800250008003504D
:100D600070B5124A1249134800F008FE124C13489D
:100D7000211C00F003FE201C00F000FE104E114D5F
:100D800000242B196159DA68301C0B4B143400F025
:100D9000F5FD642CF5D10C4800F0F0FD00F020FBCF
:100DA000011C0A4800F0EAFD70BDC046893700000A
:100DB0006E3700008D3D0000FF3D0000A13D0000AA
:100DC000BA3D000000000010C53D0000EC3D0000F1
:100DD000F0B53C4B8BB01D78002D3AD03A4B0290C9
:100DE0001B6801209B685DE001342378202BFBD039
:100DF000002B3AD0B30008336A469C500136FF2DD1
:100E000001D135E001342378202B01D0002BF9D11A
:100E1000202B02D1002323700134012E1BD12A4F35
:100E20002A4B06223B6001923D1C09E02B68029888
:100E3000196800F00EFE002808D02B6814332B60D0
:100E4000019B013B0193002BF0D132E03B681D79FF
:100E500001E0041C2E1C2378002B06D0002307225F
:100E6000B2425B41DBB2002BBFD1002E1CD000E0B0
:100E70000025154C022E05D10398154900F0E9FD17
:100E8000002801D0AE420AD823681248D96800F081
:100E900075FD23681048196900F070FD04E02368AF
:100EA000F0B29B6802A99847064B1B78002B07D12C
:100EB00003E00198011CFFF753FF084800F05EFDB6
:100EC0000BB0F0BD98020010A0020010000000104E
:100ED000F93D0000FB3D0000DA370000023E000053
:100EE00038B5041C154D0A2808D002D808281CD192
:100EF00010E00D2802D07F2817D10BE02B680022CC
:100F00001A700F4800F03AFD0E4C201CFFF760FFEE
:100F10002C6012E02A680B4B9A420ED90A48211C19
:100F200000F02CFD2B68013B06E00748211C00F077
:100F300025FD2B681C7001332B6038BD9C0200100E
:100F4000FF3D0000980100100E3E000008B503E0D0
:100F500000F0B4FBFFF7C4FF00F0D2FB0028F7D18C
:100F600008BD000008B5034A034B04481A6000F0AE
:100F700005FD08BD980100109C020010023E000013
:100F8000044B40211A680A431A60034B01221A706D
:100F90007047C04680800440A402001070B50E4B1C
:100FA000061C1B780D1C141C002B01D1FFF7E8FF59
:100FB000013E022E03D8094BB600F35800E0084B5F
:100FC0001A68012C03D1AC4014431C6003E00124D7
:100FD000AC40A2431A6070BDA40200107C3E000029
:100FE0000080005038B50F4B051C1B780C1C002BE3
:100FF00001D1FFF7C5FF0020032D11D8281C0123C4
:1010000002F0B0FA02040608074A04E0074A02E0C8
:10101000074A00E0074A1068A3401840431E984161
:1010200038BDC046A4020010FC3F0050FC3F0150F8
:10103000FC3F0250FC3F035070B50E4B061C1B7862
:101040000D1C141C002B01D1FFF79AFF013E022E4C
:1010500003D8094BB600F35800E0084B1A68012C7E
:1010600003D1AC4014431C6003E00124AC40A24314
:101070001A6070BDA4020010883E0000FC3F0050C2
:1010800038B5084B041C1B780D1C002B01D1FFF751
:1010900077FF236818229343236023681D4325604C
:1010A00038BDC046A40200101F2342091840012386
:1010B0008340181C014B9200D050704700E100E0C3
:1010C000054B3F221A60054B01221A60044B402158
:1010D0001A688A431A60704724800440D88004400C
:1010E0003882044008B5044B40211A688A431A60CC
:1010F000FFF7E6FF08BDC0463882044008B503206C
:10110000FFF7ECFD094B012252421A60084A1268AF
:10111000002A00D01A60074B1A6801321A60064A8A
:1011200000231360054A1360C04608BD08820440CE
:101130000C820440A802001004C000403CC00040E3
:1011400008B5FFF73FFD0A480021FFF799FF09485E
:101150000021FFF795FF08480021FFF791FF07489E
:101160000021FFF78DFF06480021FFF789FF08BD2A
:101170000840044000400440AC4004401440044097
:101180001C400440F7B50190FFF7DAFF574B019977
:101190001A68574B1A60002901D0564B00E0564B95
:1011A000564A04211360564B564C1A68564D0A4352
:1011B0001A60019A002A54D0544B0027544E1F60E5
:1011C000544B301C1F60391CFFF75AFF381C092193
:1011D0003A1CFFF7E3FE381C09213A1CFFF72CFFED
:1011E0004D4B802219680320114319603368072191
:1011F0008B433360336802210B43019933604B000A
:101200005B1899015B1801999B005B1843490B60BF
:10121000434B196801431960424B43491868014028
:101220001960196809200A431A60FFF73DFF226818
:1012300080239B001A43226001213C4A49421160ED
:101240002A68324913432B60394B02221A60394B0A
:1012500001221A601F601A6018681042FCD0012336
:101260000B600720FFF720FF0820FFF71DFF0A2073
:10127000FFF71AFF0C20FFF717FF0B20FFF714FFF3
:10128000236880229343236022682B4B1340236002
:1012900022682A4B134023602268294B13402360A5
:1012A0002268284B13402360019B002B03D10122AD
:1012B0001E4B52421A602B68802213432B602A680F
:1012C00080235B0013432B602A688023DB001343D9
:1012D0002B602A6880235B0113432B602A688023DC
:1012E0001B0113432B6030BFF7BDC046388204405A
:1012F00034820440BF180000FF1800003082044010
:1013000010ED00E0008204400482044004C000406C
:1013100064400440044001408080044018C0004004
:1013200014C000403CC000400FF0FFFF08820440A2
:101330007080044074800440FFFEFFFFFFFBFFFF4E
:10134000FFEFFFFFFFF7FFFF08B5FFF71BFF08BD2B
:1013500000B5064B1A6801321A601B68013303D1CD
:10136000034B1A6801321A6000BDC046B00200107B
:10137000AC02001000B5074B98420AD8064A002379
:101380001360064A01381060054A1360054B0722B6
:101390001A6000BDFFFFFF00B002001014E000E083
:1013A00018E000E010E000E000B50C4A13680028E7
:1013B00000D10120C1438B4204D809E01168814269
:1013C000FCD301E0591C081811689942F6D203E0D9
:1013D0001168C91A8142FBD300BDC046B00200109B
:1013E00010B5064BFA211868054B89001C6802F0FD
:1013F000CDF8044B5C43201810BDC046B00200106D
:10140000AC02001037894100034B01221A60034BE4
:101410001A6801321A60704700C00040B402001020
:10142000034B01221A60034B1A6801321A6070479D
:1014300000000140B8020010034B01221A60034B68
:101440001A6801321A60704700400140BC02001067
:10145000034B01221A60034B1A6801321A6070476D
:1014600000800140C002001000B5002803D1044BE9
:1014700001221A6003E0012801D1024B186000BD6F
:10148000044001400480014000B5002802D1044B13
:10149000186004E0012802D1024B00221A6000BD4E
:1014A000044001400480014010B5041C002906D10D
:1014B000164B96201968C00002F068F8011C002C39
:1014C0000FD1134B80221868920002431A60114B0F
:1014D00003221C60104B1960104B1A608022D2024C
:1014E00011E0012C11D10A4B80221868D20002436E
:1014F0001A600B4B00221A600A4B032219600A4B38
:101500001A6080221203094B1A6010BD78800440D3
:1015100080800440BC02001018400140144001408B
:10152000C0020010188001401480014000E100E07A
:1015300008B5184B1A680E231340062B0DD1164B15
:101540009E221B68DBB2134204D0144A5360144B32
:101550001B681EE0D9071CD501E0042B05D1104BF8
:101560001868C0B200F0BBF813E00C2B06D10B4B8F
:101570008022596852000A435A600AE0022B08D1BF
:10158000054B1A68054B910601D5002200E00122A7
:101590009A6008BD0880004014800040C40200101A
:1015A0000080004000487047C402001070B52B4C0A
:1015B0002B4B80229203DA6700219022061C201C0C
:1015C00000F014FA0023A36000F072F8254B072501
:1015D0001A68254CAA431A60196801221143196040
:1015E000224B1968A9431960196811431960204BEF
:1015F000802118684901014319601E4B1E481A607A
:101600008322226019681D4B1B68584301F0BEFFFE
:10161000311C000901F0BAFF1949030A194A0B608D
:10162000C0B2032310602360174B1D60174B18686E
:1016300060201C680440602CFBD101E0146800E0CD
:1016400001201C680442F9D1044B01221A70104B8E
:10165000802292031A6005230B6070BDC402001043
:1016600004E100E0A44004400C800040A840044095
:101670008080044098800440001BB70078800440BC
:10168000048000400080004008800040148000403A
:1016900000E100E000B5044A202311681942FCD0A3
:1016A000024B186000BDC04614800040008000401E
:1016B00008B5FFF777FF0023437308BD08B5FFF7B0
:1016C00071FFC27B031C8218107CDA7B7F21013200
:1016D0000A40DA735A7B013AD2B25A7308BD10B588
:1016E000041CFFF75FFF837B7F22C3181C74837B7E
:1016F000013313408373437B0133DBB2437310BD6B
:1017000008B5FFF74FFF407B431E984108BD30B539
:10171000002402E00570013401301D5D002DF9D177
:10172000121B131C02E00170013B0130002BFADC9C
:10173000D043C0170240A01830BDF8B5051C0F1CDF
:101740001E1C541E092B01D800240FE0181C0A216E
:1017500001F01CFF221C031C391C281CFFF7EDFFA5
:10176000041C2D1805E02F7001340135013A002AC0
:10177000F9DC301C0A2101F04DFF30312970601C6A
:10178000F8BDF8B50C1CD9175F18061C4F40551E44
:10179000092F12D9381C0A21002B03DA01F0F6FEBA
:1017A000434202E001F0F2FE031C211C2A1C301C03
:1017B000FFF7E7FF041C351813E0002B00DA951E35
:1017C000002201E0B4540132A91A0029FADCEC43EA
:1017D000E4172C403519002B03DA2D232B7001342C
:1017E0000135381C0A2101F015FF30312970601CC9
:1017F000F8BD73B5069E041C1D1C3009531E00283D
:101800000AD000901A1C201C2B1CFFF7F2FF241892
:1018100005E0217001300134013A002AF9DC0F2380
:101820001E40092E01D8303604E0002D01D0373695
:1018300000E057362670013076BDF0B585B0041C47
:101840000F1C002801D00021017000256BE0252924
:1018500003D021700132013405E05178252904D1EB
:1018600021700232013401355DE0302903D00132AC
:101870000292202101E002320292029E9C463278BE
:101880002D3A50424241B6180296002205E00A2342
:101890005A438218303AD2B201363078031C303BBA
:1018A000092BF4D90296AE186346BE4201D97A1BC1
:1018B000D2B269280ED006D863282CD0642809D06B
:1018C00058283ED119E075280AD078280FD07328FF
:1018D00037D11AE01E1D201C1B68FFF752FF04E0E1
:1018E0001E1D201C1B68FFF728FF331C17E01E1D60
:1018F0001B68201C0093002304E01E1D1B68201C95
:1019000000930123FFF775FFEFE71E1D201C1B68E6
:10191000FFF7FDFEE9E71A68012022700433029AFE
:10192000241801322D181178BD4201D200298ED120
:101930000023BD4201D2237005E0013C2370013D2C
:1019400001E001256D4205B0281CF0BD10B50C1C4E
:10195000131C6421221CFFF770FF10BD00B5031C8F
:101960009BB00A1C01A8191CFFF7F0FF632800DDDB
:10197000FEE701A800F09CF81BB000BD0FB407B54E
:1019800004A901C90191FFF7E9FF03B008BC04B045
:1019900018470EB403B503AA02CA0192FFF7D6FF97
:1019A00002B008BC03B0184770B50323041C1842EA
:1019B00005D10D1C041C194201D1934201D300230F
:1019C00011E0131C40CD043B40C4032BFAD8141F74
:1019D000A4080134A400032309191A400419EEE7EE
:1019E000CD5CE55401339342FAD170BD30B50B04A0
:1019F0000D061D430D430B021D430323041C93429C
:101A00000DD218420BD1131C043B20C4032BFBD86E
:101A1000141FA4080134A40003231A40041900234E
:101A200001E0E15401339342FBD130BD00B5002306
:101A300000E00133C25C002AFBD1181C00BD00B5D8
:101A4000031C01E0013101330A781A70002AF9D130
:101A500000BD00B502E00130002B06D00A78037803
:101A600001319342F7D0981A00E0181C00BD000025
:101A700008B5FFF751F90B48FFF77CFCFFF780FA38
:101A8000FFF730FB96200002FFF790FDFEF7E6FE21
:101A9000FEF7D2FE044A0548111CFFF76FFFFFF75F
:101AA00061FA08BDE02E0000FF3D0000943E0000FA
:101AB00010B5041C02E00134FFF7ECFD207800288B
:101AC000F9D110BD00B50B4B984201DD0A4BC0188F
:101AD0000A4A8310D35C03220240082152008A1A6A
:101AE00093401A1CC0239B001A40054B1B5C101C22
:101AF000184300BDFF17000000F8FFFFC23E0000C2
:101B0000C244000008B54018511A013101F0EEFD41
:101B100008BD08B5801889189A1A0132FFF744FFEA
:101B200008BD000030B5B14B87B0D96EB04D4A1E2C
:101B300091416A46D175A96A1A1CC806400F01383E
:101B4000062807D801F00EFD040C1F1217191C00FF
:101B5000022409E05A6E16329200D3581C1C15E07C
:101B60005B6E16339B00D45800230FE09B6DD46D41
:101B7000A3420ADC0AE0022403E00C24032305E06C
:101B80000D24231C02E00D24EEE70D242C614811E6
:101B90001F2800D922E16A461732944901F0ECFC73
:101BA0002000220028002A002D002F0038004000CD
:101BB0004400490051005F0067006F007700850016
:101BC0009300A200B400C300D500D300E300E600F8
:101BD000E900F100010105010F01110113011901D3
:101BE000081C00E08348191C221CFFF78BFFF5E05E
:101BF0008148F8E70A1C0E3203E07E4809E00A1C1F
:101C00001C32081C111C1A1C231C01F0FDF8E5E015
:101C10007948011C0E391A1C231CFFF77AFFDDE0FE
:101C20007448011C0E31EEE70A1C1C32081C111C02
:101C3000F1E70A6E1020002A00D00A200A1C0E329A
:101C400006E00A6E1020002A00D00A200A1C1C326E
:101C500000946C46173402900194081C51E0012056
:101C60001070086E1022002844D00A2242E00A6E4A
:101C70001020002A00D00A200A1C0E320EE001209B
:101C80001070086E1022002855D00A2253E00A6E08
:101C90001020002A00D00A200A1C1C3200946C4636
:101CA000173402900194081C78E00A6E1021002A73
:101CB00000D00A21504A68461730019002910094E2
:101CC000101C111C1DE00A6E1020002A00D00A20F2
:101CD000494A00946C46111C173402901C39019437
:101CE000101C0EE0096E012010701022002900D097
:101CF0000A22414968461730019002920094081C5C
:101D0000002201F08BF869E00A6E1020002A00D052
:101D10000A20394A00946C46111C173402901C3971
:101D20000194101C3AE0096E012010701022002965
:101D300000D00A2230496846173001900292009480
:101D4000081C00222AE0012010700A6E1021002ACF
:101D500000D00A21284A6846173001900291009469
:101D6000101C00211AE0009222481CE00092224838
:101D700019E00A6E1020002A00D00A200A1C1C322A
:101D800006E00A6E1020002A00D00A200A1C0E323B
:101D900000946C46173402900194002001F067F81B
:101DA0001CE00092081C002104E00D1C1C35081CDE
:101DB0000092291C1A1C231C01F0B4F80EE0081C28
:101DC00002E00C4800E00C48191C221C01F0C3F88A
:101DD00004E0081C221C191C01F0C8F86B46DA7DCF
:101DE000024B07B00120DA6630BDC0468C040010FB
:101DF000281300109A040010A804001010B506491A
:101E00000B1C88331A68141C1E34A4006050013265
:101E100003210A401A6010BD8C040010054B0320FA
:101E2000191C88310A68013A02400A601E32920089
:101E3000D05870478C040010F8B5114D2C1C8C3410
:101E400020680130FFF73EFE0E4B0122D8629F6AE8
:101E5000AB6E061C02409A4210D1830703D420685F
:101E60000230FFF7CBFFFF239B001E40B601BF10DF
:101E7000044B8C35374301222F60DA600220F8BD15
:101E80008C0400102813001030B50C4B0C489A6AD3
:101E9000031C8C331C68D3059B0E910500D5403B79
:101EA000856E921001210A40AA4204D1E3188C30B9
:101EB0000360024BD960012030BDC04628130010DA
:101EC0008C04001008B5084B5A1CD07F9A1CD27F96
:101ED000000112021043DA7F0333DB7F10431B0340
:101EE0001843FFF78BFF08BD8C04001038B5FFF7CF
:101EF00095FF064903230F22051C5C18154001338A
:101F000025770011072BF7D138BDC0468C0400108F
:101F100008B5FFF783FF034B01228C331860024B97
:101F2000DA6008BD8C0400102813001010B5064CB0
:101F3000A36E002B06D0FFF771FF044B8C340122F7
:101F40002060DA6010BDC0468C0400102813001019
:101F500010B5064CA36E002B06D1FFF75FFF044BB4
:101F60008C3401222060DA6010BDC0468C04001061
:101F70002813001008B5124B1B68002B00D098479F
:101F8000104B5A69002A15DD012A07D1DA69002AA7
:101F900004D09A610022DA610A225A615B69032245
:101FA000191C91430A1E02D0074A0121D166054A35
:101FB000013B5361044B90331A68024B5A6208BDCF
:101FC00054030010281300108C04001000B5064BB9
:101FD0005A69002A07DD9A690F21044B1140D9770D
:101FE00012110133DA7700BD281300108C040010A1
:101FF000044B597F9A7F090112020A43197F0A4351
:102000005A6770478C04001030B50B1C093B012B3C
:102010000FD8084A00239C18257FC45CA54205D030
:10202000054B08395A681143596002E001330E2B01
:10203000F1D130BD8C0400102813001000B5082920
:102040000DD0192911D1427808231A4202D000225A
:10205000027002E00F2303700723437005E00023A2
:102060001A1CC25401330E2BFBD100BD10B50E4B10
:10207000596F002802D00F22914301430E244C4394
:1020800059679C33E418094B1B68292B02D0201C8C
:10209000FFF7D4FF044A0023E05C99180133087766
:1020A0000E2BF9D110BDC0468C040010281300106F
:1020B00070B5124B0F225C6F944304435C67104B66
:1020C0001B68292B01D0082C17D00E2565430D4E17
:1020D000211CAD19281CFFF797FF9C3E00239A197D
:1020E000127FEA5401330E2BF9D1054B1B68292BC3
:1020F00003D0281C211CFFF7A1FF70BD8C04001029
:10210000281300102805001038B5104B104D1B681F
:10211000292B02D06B6F082B17D0696F0E244C430C
:102120009C356419201CFFF76FFF9C3D00235A1952
:10213000127FE25401330E2BF9D1044B1B68292B7B
:1021400003D0696F201CFFF779FF38BD28130010FA
:102150008C04001010B50D4C631CD87FA31CDB7FD2
:1021600000011B021843E37F1843E31CDB7F1B03C2
:102170001843FFF7A7FC0F23021C1A402277021115
:10218000134000126377A07710BDC0468C04001086
:10219000044B5A6E16329200D258121A51424A41DA
:1021A000DA6670478C04001000B5064B5A6E163282
:1021B0009200D1580139D150002901DA0D21D150B6
:1021C00000BDC0468C04001000B5064B5A6E163296
:1021D0009200D1580131D1500E2901D10021D150A6
:1021E00000BDC0468C04001000B5094B5A6E163273
:1021F0009200D2580D2A03D11A1C2932127805E018
:102200009A18507F117F0001021C0A435A6500BDD5
:102210008C04001010B5084B0F245A6E1632920031
:10222000D1585A6D58181440013104770D2902DC39
:102230005B1812111A7710BD8C04001030B50F4BCB
:102240005A6E596D16329200D2580D2A07D11C1CB5
:1022500029342478F02008402043586507E0981876
:10226000447F057F24012C435C650B114377034BAE
:102270009A180F231940117730BDC0468C04001006
:1022800008B504480022011C1C390D23FFF741FC4E
:1022900008BDC046C404001008B504480022011C53
:1022A0001C310D23FFF735FC08BDC046A804001003
:1022B00008B504480022011C1C310D2300F0A4FDC8
:1022C00008BDC046A804001008B504480022011C3F
:1022D0000E390D23FFF71DFC08BDC046B6040010E3
:1022E00008B504480022011C0E310D23FFF711FC34
:1022F00008BDC046A804001008B504480022011C0F
:102300000E310D2300F080FD08BDC046A80400106A
:102310000C4A0023111C46310B70111C47310B7005
:10232000111C48310B70111C49310B70111C4A31C2
:102330000B70111C4B310B70111C4C314D320B705A
:10234000137070478C04001000B5074A011C042369
:1023500000208A1804E0D11846310978400008436B
:10236000013BF8D200BDC0468C04001030B5074ACE
:1023700000238918012206E0CC18051C46341540BC
:10238000257040100133042BF6D130BD8C040010B1
:1023900038B50020FFF7D8FF084C051C0021207F2E
:1023A000FFF7E4FF25770420FFF7CEFF0421051C8B
:1023B000607FFFF7DBFF657738BDC0468C040010F7
:1023C00010B50020FFF7C0FF034C20770420FFF773
:1023D000BBFF607710BDC0468C04001010B5054CE3
:1023E0000021207FFFF7C2FF607F0421FFF7BEFFBF
:1023F00010BDC0468C04001010B5094C231C8C3352
:1024000018680130FFF75EFB064B021CD8620F23F1
:102410001A4022770211134000126377A07710BD93
:102420008C0400102813001010B5094C0021201C4A
:102430000D22FFF767FB201C0E3000210D22FFF755
:1024400061FB201C1C3000210D22FFF75BFB10BD3F
:102450008C04001010B50C4B00211A1C187F1C783E
:1024600001312043187701330E29F7D1936E002BE9
:1024700008D0064B1B690D2B04D1137F111C293189
:102480000B70537310BDC0468C040010281300104D
:1024900010B50C4B00211A1C1C7F1878013120400C
:1024A000187701330E29F7D1936E002B08D0064B15
:1024B0001B690D2B04D1137F111C29310B70537331
:1024C00010BDC0468C040010281300107FB50023F7
:1024D0000C4A0D251C1C1118097F01306E469955B8
:1024E000C60F8542664176420133111C30400E2BE7
:1024F000F1D100236C46185DCA18013310770E2BFA
:10250000F8D17FBD8C04001010B5074B5A6E1632FF
:102510009200D1585C1801392077D150002901DA96
:102520000D21D15010BDC0468C040010034A002379
:10253000111C943198320B60136070478C040010AA
:10254000034B012194331A684A401A607047C04611
:102550008C040010044A002313678C321360034B71
:102560000122DA607047C0468C0400102813001066
:1025700008B59A4B0F20996A994A8B101840891117
:10258000013852560E2800D9C1E000F0EBFF0811C7
:102590001A2327C02EC0C037C0C0C03B3F00002A4E
:1025A00000DAB4E08F4B9A18403200239371A9E00F
:1025B000002A00DAABE08B4B01209A184032907170
:1025C000A4E0002A00DAA2E0864B9A184032927901
:1025D000DA6697E0081CFFF797FF93E0002A00DA1D
:1025E00095E0101CFFF7D4FD8CE0002A00DA8EE0A5
:1025F0007C4B596E16318900CA5083E0081CFFF7E6
:1026000057FD7FE0081CFFF731FD7BE0002A00DA70
:102610007DE0101CFFF75AFF74E0724B01209833E5
:10262000186073E0FFF7E0FD6CE0FFF793FF69E0EF
:10263000FFF726FE66E0FFF7EDFD63E0694B002241
:102640005A665FE0FFF728FE5CE0FFF7F7FD59E010
:10265000644B0120586659E0FFF72AFE52E0FFF76D
:10266000CBFE022052E0FFF72FFE4BE0FFF72AFCE3
:1026700048E0FFF735FE45E0FFF7D6FE42E0FFF702
:1026800035FC3FE0FFF738FE3CE0FFF79FFC39E008
:10269000544B00221A6635E0FFF7AAFC32E0514B9A
:1026A0000120186632E0FFF741FF2BE0FFF72CFD19
:1026B00028E0FFF745FF25E0FFF74CFD22E0FFF79C
:1026C0008DFE1FE0FFF732FC1CE0FFF7C3FE19E0B0
:1026D000FFF776FE16E0FFF73BFC13E0FFF7D8FEAE
:1026E00010E0FFF715FE0DE0FFF744FC0AE0FFF7EE
:1026F0005BFD07E0FFF74CFE04E0FFF765FD01E03E
:10270000FFF706FC012001E00120404208BD982BA4
:10271000BED03EDC382B9BD01DDC1C2B00D187E7C4
:102720000CDC0C2B00D178E702DC002BEAD0EBE7C5
:10273000162B00D176E7182BE6D176E7282B00D1AF
:102740007CE702DC262BDFD175E72C2B00D179E763
:10275000362BD9D179E7662B00D18AE70CDC4C2BDC
:1027600000D17CE702DC3C2BCED175E7562B00D1A3
:1027700079E75C2BC8D179E76C2B00D17FE702DCCD
:10278000682BC1D178E7762B00D17BE7882BBBD1B2
:102790007BE7E62B00D19BE726DCC82B00D188E73E
:1027A0000CDCA82B00D17AE702DC9C2BACD173E7C0
:1027B000B82B00D177E7BC2BA6D177E7D62B00D179
:1027C0007DE703DCCC2B00D09EE775E7D82B00D14A
:1027D00078E7DC2B00D097E777E7C0462813001096
:1027E000C25C00008C040010F32B00D17CE70EDCEF
:1027F000EC2B00D172E703DCE82B00D084E76AE71A
:10280000F12B00D16DE7F22B00D07DE77AE7F62BB4
:1028100000D16FE703DCF52B00D075E767E7F72BF6
:1028200000D16AE7F82B00D06EE769E738B5184C9D
:10283000231C8C331868FFF745F9211CE26E903198
:10284000144B0D68A2660022E2660135DA600322AD
:1028500098620D601040251C1C1C022809D0904273
:102860000AD0012802D0FFF783FE07E0FFF7E4FA61
:1028700004E0FFF757F901E0FFF706FB002806DD4B
:10288000E368002B03D18C352B681B182B6038BDF7
:102890008C04001028130010034B0122DA660F226B
:1028A0009A775A771A7770478C04001010B5054C48
:1028B0000549201C00F01AFFFFF7EEFF01236366B5
:1028C00010BDC0468C0400109C0E000000B5074BE4
:1028D00000201B680F2B08D1054B1A78824204D1C7
:1028E0001868044B1840431E984100BD6400001056
:1028F0008C04001000FFFF0038B5164B1A1C9832EC
:102900001268002A04D0144B1D6801231D4001E009
:1029100094331D68114CA3689D4202D16268002A5D
:1029200016D0002D02D1002B0AD111E00C4B1B68F0
:10293000002B02D06168281C98470023636006E0E2
:10294000074B1B68002B02D0281C291C9847A56048
:1029500038BDC0468C04001074030010281300100A
:102960006C03001013B5002300930193244B1B68E4
:10297000002B02D0684601A998472249009B08789D
:10298000214A00280CD0002B02D00223137035E01E
:102990001378013BDBB21370002B2FD10B7009E0D1
:1029A000002B0CD11378002B28D0013BDBB2137025
:1029B000002B23D1154A1360154A13601EE01449F9
:1029C0000968581A44426041400010701148446937
:1029D000021C002C04D08B4202D10A2343610DE07B
:1029E00000290BD10A21516101999361D161084AF3
:1029F0001360064B02221960034B1A7013BDC046C8
:102A00005C03001078030010600300105C130010DA
:102A1000581300102813001008B5FFF7A3FF08BDD6
:102A200010B5094C20600948016009490A60094A4B
:102A30001360094B029A1A60084B039A1A60084AFD
:102A4000084B1A6010BDC0466C0300105C030010F8
:102A500068030010640300105803001064000010A5
:102A6000192A00005403001008B5084B084A1968D9
:102A700012688A1A1A6006D5FA2252001A60054BAB
:102A80001A6801321A60FFF737FF08BD68000010AE
:102A90005803001074030010F7B50E1C0E21051C1E
:102AA000019200F023FE1A4B03240C279E420FDDF7
:102AB00009236B7301232B7328E0301C0A2100F0DB
:102AC00009FE301C29550A2100F0AEFD0134061C18
:102AD000002E06D0E30F0022A7425341DBB29342FF
:102AE000EBD1019AA31A033B2B70621B2B1C01E054
:102AF000195D5973013BD1180229F9D10F231C1B11
:102B0000002301E0013C2B55032CFBDCF7BDC04644
:102B1000FFC99A3B38B50C4B01221A700B4B0222AD
:102B20001A700B4D0B4C08E01868884208D01B68DF
:102B30002360FFF799FFFFF715FF2B682168024A12
:102B400010780028F0D138BD780300106003001021
:102B500064030010700300104278037812011A43D6
:102B6000C37881781B010B43D01A7047F0B5224A15
:102B7000224B0F1CD45CE8235B00D35C24011C4374
:102B80001F4BE121D35C4900515C1B0185B00B4315
:102B90000293E9235B000390D55C002C02D18024D2
:102BA00007256400174E301CFFF7D6FF0299421C20
:102BB000631A802149000C1B07214D1B0398124901
:102BC00001950094FEF7E5FE00233B704125023E8F
:102BD000381CFEF72BFF3C18301CFFF7BDFF2A1CEA
:102BE000031C0A49201C0135FEF7D3FE023E462D88
:102BF000EED105B0F0BDC0468C040010D10100003C
:102C0000C301000058060010D25C0000DF5C000029
:102C100030B53D4B3D4C1A1C9432126891B0A06106
:102C2000E161002A17D118280BD1C32909D1384AEC
:102C300012680F2A05D1181C38300E21162200F018
:102C4000CFF8A369182B04D1E369332B01D100F02D
:102C500071F8FFF721FE0A2363612B4C01232D4DF0
:102C600023678C34FFF7E2FD2368AB4218D006DC03
:102C7000294A934219D0294A93422ED106E0284A84
:102C8000934208D0274A934227D117E0204B1B6874
:102C90000B2B22D10DE01E4B1B680C2B1DD108E025
:102CA0001B4B1B680F2B18D103E0194B1B68102B13
:102CB00013D1FFF721FEFDF70AFA0EE0144B1B6853
:102CC0000F2B0AD1684608A9FFF750FF164B1B6867
:102CD000002B02D0684608A99847144B1A68144B79
:102CE00010681968884205D012681A60FFF7BCFEA8
:102CF000FFF738FE044B1B6F002BB3D1FFF7FCFD31
:102D0000FFF708FF11B030BD8C040010281300102D
:102D100064000010790D00006A0C0000130D000023
:102D2000990D00006527000068030010640300107F
:102D30007003001070B5254C23681D68FFF7EAFE8C
:102D400023681A689542FCD01E68FFF7A5FD204B4A
:102D50000A22204C5A6118229A611522DA61231C3A
:102D6000903300221A60FFF797FD01232367643632
:102D7000164C194D0AE0FFF759FD23682A681968B7
:102D8000914203D01B682B60FFF76EFE23681B681F
:102D90009E42F0D10F4D18202B1C90331C6800214F
:102DA000FFF736FF0D4B60001968001900F03CFC7E
:102DB0003835011C0422281CFFF76EFE044B182234
:102DC0009A610022201CDA6170BDC04664030010C5
:102DD000281300108C04001070030010580300101A
:102DE000F0B501240DE005780B1C254006E0C65C1B
:102DF000ED0077083D43C554351C2540013BF6D511
:102E0000013A002AEFDCF0BD30B504E0845C8D5C53
:102E100085548C5401329A42F8DD30BDF7B5099DD6
:102E20000AAC2678089F2C7894461D1C002A0DD1E8
:102E300018E063465B5D4A5DD218131901920024C5
:102E4000B34201DB9B1B012443550135BD42F0DD3C
:102E50000AE0CA5C12190024B24201DB921B012471
:102E6000C2540133BB42F4DD099B1C70F7BDF7B5BA
:102E7000099E0AAC2778089D347800282FD00029B5
:102E80002AD01E1C9446002A0ED1013F18E063464A
:102E90009B5D8A5DD21A131B00240192A34201DAC2
:102EA000DB19012483550136AE42F0DD37E0CA5C00
:102EB000121B0024561C01D13A1C0124C2540133B8
:102EC000AB42F4DD2BE0D15C49420C1B211E01D04A
:102ED000E1190124C1540133AB42F4DD1FE00029A4
:102EE0001BD0181C002A06D10EE00E5C135C0130CA
:102EF000F31A1C1BE40FA842F7DD10E0CA5C013393
:102F0000141B013462425441AB42F7DD07E0D15C4F
:102F1000013349420C1B611E8C41AB42F7DD099A1B
:102F20001470F7BD70B5049D01242C70141C002989
:102F300005D10BE0065D0A5D96420BD101349C423F
:102F4000F8DD05E0815C002904D101329A42F9DD07
:102F500000232B7070BD00B503E043185B78435429
:102F600001319142F9DB0023435400BD00B504E078
:102F70008318013B1B788354013A8A42F8DC002312
:102F8000835400BDF0B5114B1A785B78825C1A400F
:102F900000D040220E4C0F49231C261C04C32C36A3
:102FA00000221A6001240A1C123117785578C75D77
:102FB0003D4202D01F6827431F60023264008A42EC
:102FC000F3D10433B342EBD10020F0BD6101001016
:102FD000F0140010AD00001030B512234B43334AFB
:102FE0000131D3188A0051181A785C78825C144237
:102FF00004D02F4A5F245218947054709A78DC7869
:10300000825C144204D02A4A7C2452185332147031
:103010001A795C79825C144204D0254A7C245218C7
:10302000A33214709A79DC79825C144207D0204C68
:103030005F226418251CA235A1342A7022701A7AE6
:103040005C7A825C144204D0194A7C245218A03263
:1030500014709A7ADC7A825C144204D0144A7C247C
:103060005218503214701A7B5C7B825C144207D079
:103070000F4C5F226418251C523551342A7022707F
:103080009A7BDC7B825C144204D0094A2E245218BD
:10309000A43214701A7C5B7C825C134204D0044B13
:1030A0005918F43127230B70002030BDAD000010FB
:1030B00060130010F8B52D4C071C0025201C2021A2
:1030C0004F22FEF793FC002D04D0221C7C233932C2
:1030D00023701370231C4F330021013519705034B5
:1030E000052DEBD1214B2D22181C38300270181CF5
:1030F00037300270A1209A705A7040005F221A5433
:103100001B481A54A320400019541A4908784978DA
:10311000385C014204D0191C533152330A701A70C2
:103120000024211C381C0134FFF756FF0A2CF8D16B
:10313000114D124E00242B786A78FB5C1A4201D0A4
:10314000315905E03059FEF771FC0D49091A0A3171
:103150000C48043400F0D4FA0235242CEBD10A498F
:10316000084800F0CDFA0520F8BDC04660130010F5
:1031700041010000610100106C000010800000108F
:1031800063010010A0140010E75C0000F0B585B0EA
:1031900001900027FDF750FB6A4C3E1C6A4A7542BD
:1031A000754113687D19012B05D168480D210C224A
:1031B000FDF702FC02E0002B00D1CDE0002303AAC2
:1031C000537023687F210B405C2B00D198E02ADCF0
:1031D000382B00D18EE013DC072B6AD006DC022BE3
:1031E00000D193E0062B00D0B6E041E0212B00D1C6
:1031F00084E0232B00D187E01C2B00D0ACE081E0E1
:103200004F2B4ED007DC3F2B62D0402B62D0392BA6
:1032100000D0A1E064E0542B76D05B2B3FD0502B44
:1032200000D099E06AE0732B66D010DC662B3AD0B0
:1032300005DC5E2B56D0622B00D08DE062E06F2B58
:103240003BD0712B52D06D2B00D085E02DE0792B37
:103250004AD006DC762B4BD0772B3DD0742B7BD11C
:1032600046E07D2B23D07F2B25D07C2B74D135E0FD
:1032700031231370022E4BDD231C083B1B681940C1
:10328000542908D0032E43D0231C0C3B1A687F23FB
:103290001340542B3CD14C2203AB1A7038E032233C
:1032A00035E0332333E0342331E035232FE0362378
:1032B0002DE037232BE0382329E039231370062E25
:1032C00026DD231F1B6819404723232920D11EE038
:1032D00030231CE02D231AE0412318E0422316E09E
:1032E000432314E0442312E0452310E046230EE07C
:1032F00048230CE04C230AE0502308E0522306E068
:103300004F2304E0552302E04E2300E049231370CD
:10331000ADB203A8291C0022FDF7C2FB23681A06E0
:1033200005D5E91D89B20A480022FDF7B9FB2368DB
:10333000DA0572D50735A9B206480022FDF7B0FBC1
:103340006BE0C046F0140010700100104E39000010
:103350003A3E0000EF5C000023680122134206D0D1
:10336000A818C0B2002107220223FDF705FB23683D
:103370000222134205D0A81DC0B200210623FDF78A
:10338000FBFA236804210B4205D0A81DC0B202221B
:103390000623FDF7F1FA236808210B4205D0681CCB
:1033A000C0B207220223FDF7E7FA2368DA0606D542
:1033B000681CC0B2042102220623FDF7DDFA23684F
:1033C0009A0606D5681CC0B2002102220623FDF72A
:1033D000D3FA23685A0606D5681CC0B20421072216
:1033E0000223FDF7C9FA23681A0607D5281C0930FD
:1033F0000222C0B20821131CFDF7BEFA2368DA05C9
:103400000BD5EDB2281C0930C0B20B210A35FDF7EF
:103410009DFAE8B20A21FDF799FA013604340C3717
:103420000B2E00D0BAE61B4803210622FDF7C4FA92
:10343000194D1A4E1A4F0024019A2B78D35C6A78E2
:103440001A4205D0A3009859395D0922FDF728FBDF
:1034500001340235092CEFD1FFF738FA002814D0D7
:1034600006240321201C00F0DFF80321C5B2201C34
:1034700000F030F9281CC9B2FDF768FA092C01D117
:103480000B24EEE701340E2CEBDDFDF7DFF905B080
:10349000F0BDC046093800006C0000107401001037
:1034A000A400001070B5041CFFF76CFD201CFFF792
:1034B0006DFE0A4B1B78002B0ED0201CFFF7FAFD87
:1034C000074CC8235B00074EE518211C301C503404
:1034D000FEF754FAAC42F8D1002070BD7903001019
:1034E00060130010DA37000008B5002805D0FDF79A
:1034F00082F90748FFF7D6FF08E0FDF784F9054B8E
:103500001B78002B02D00448FEF738FA08BDC046ED
:10351000A605001079030010F15C000000B5FEE77D
:1035200000B5FEE708B50A4B0A4A0B4903E01078DC
:103530000132187001338B42F9D3084B084900223D
:1035400001E01A7001338B42FBD3FCF725FFFEE745
:1035500000000010485D0000980100109801001064
:103560001C15001002B4714649084900095C490065
:103570008E4402BC7047C04603B4714649084000FF
:103580004900095A49008E4403BC7047002934D0D1
:103590000123002210B488422CD301242407A14225
:1035A00004D2814202D209011B01F8E7E400A142E2
:1035B00004D2814202D249005B00F8E7884201D37D
:1035C000401A1A434C08A04202D3001B5C08224355
:1035D0008C08A04202D3001B9C082243CC08A042C6
:1035E00002D3001BDC082243002803D01B0901D0B2
:1035F0000909E3E7101C10BC7047002801D0002027
:10360000C04307B4024802A14018029003BDC0465F
:10361000D90000000029F0D003B5FFF7B9FF0EBCB8
:103620004243891A1847C046002941D010B4041CEF
:103630004C40A44601230022002900D5494200281D
:1036400000D5404288422CD301242407A14204D251
:10365000814202D209011B01F8E7E400A14204D231
:10366000814202D249005B00F8E7884201D3401A48
:103670001A434C08A04202D3001B5C0822438C086A
:10368000A04202D3001B9C082243CC08A04202D3D4
:10369000001BDC082243002803D01B0901D00909C4
:1036A000E3E7101C6446002C00D5404210BC704774
:1036B000002806D003DB0020C043400801E0802042
:1036C000000607B4024802A14018029003BDC0469C
:1036D000190000000029EBD003B5FFF7A7FF0EBCCF
:1036E0004243891A1847C0467047C04600B50029B2
:1036F00005D000230139037001300029FAD100BD43
:10370000F8B5041CA30719D1231C04CB0F4D104E90
:1037100050199043021C201C32420FD1181C0B4F31
:1037200004CBD5199543354208D1181C074F04CB5B
:10373000D51995433542F1D000E001300378002BD4
:10374000FBD1FEF77CF9201CF8BDC046FFFEFEFE53
:103750008080808053455249414C20434F4E534F07
:103760004C450025732072656164790D0A00444D53
:1037700031314343000D0A4279652E2E2E0D0A0089
:1037800025732025732025730056414E494C4C412A
:10379000005633002578000D0A25303278202000AD
:1037A0000D0A413A2000202025633A20000D0A4DE1
:1037B0003A20002020473A20253032780D0A005761
:1037C000616974696E6720666F7220646174612E2E
:1037D0002E2E0D0A00526561642025730D0A004FDC
:1037E0004B004641494C454400656E61626C65641E
:1037F0000064697361626C6564004C4344206465D5
:103800006275672025730D0A00030300000003039F
:10381000005C0003030C000C03037C287C03037C86
:10382000447C030324104803032854080303000CBA
:103830000003033844000303443800030320100846
:10384000030310381003038040000303101010031B
:103850000300400003032010080303384438030327
:10386000007C000303645448030344542803031CEE
:10387000107C03034C5424030338542003030474C2
:103880000C03032854280303085438030300500092
:10389000030380500003031028440303282828034F
:1038A0000344281003030454080303384C5C030347
:1038B00078147803037C5428030338444403037CBE
:1038C000443803037C544403037C14040303384446
:1038D0003403037C107C0303007C00030320403C82
:1038E00003037C106C03037C404003037C087C03CF
:1038F000037C047C03037C447C03037C14080303E3
:1039000038447803037C14680303485424030304F5
:103910007C0403037C407C03033C403C03037C2089
:103920007C03036C106C03031C601C030364544C85
:1039300003037C440003030810200303447C0003BA
:1039400003080408030380808003030408000007C1
:10395000080400000000BF01BF01090500000700C6
:103960000700070007130A00002000E400FC003FE6
:1039700000E700FC003F002700040F0800000C01D6
:103980001E01FF03FF032201E201C2190D00000E18
:10399000001F0011019101FF007E00FC00FE0113D9
:1039A000011101F001E0140A0000EE00FF01110115
:1039B0001101BF01EE00E00130011001050300001C
:1039C0000F000F0A050000F800FE03070701040BB3
:1039D000060000000001040707FE03F80F080000BE
:1039E00000000A000E001F001F000E000A1109004F
:1039F00000100010001000FE00FE0010001000106B
:103A0000080400000004800780030D070000100078
:103A100010001000100010001008040000000080CA
:103A20000180010D07000C000FC003F0003C000FE7
:103A300000030F080000FE00FF0101010101010168
:103A4000FF01FE10080000000002010201FF01FF5B
:103A50000100010001100800008601C70161012179
:103A60000131011F010E010F0800008200830111C6
:103A70000111011101FF01EE1109000030003800B1
:103A80002C002600FF01FF012000200F080000800D
:103A9000009F011F0111011101F101E10F08000058
:103AA000FC00FE010B0109010901F901F00F0800FA
:103AB0000001000100C101F1013D000F00030F08EA
:103AC0000000EE00FF01110111011101FF01EE0FD5
:103AD0000800001E003F0121012101A101FF007E1D
:103AE0000804000000008C018C01080400000004A0
:103AF0008C078C0312090000200070005000D800D1
:103B000088008C01040104011109000048004800EC
:103B100048004800480048004800481109000004D7
:103B20000104018C018800D80050007000200D07AE
:103B3000000002000300B101B9010F0006190D00D9
:103B400000F800FC010603FB06FD0505050505FD63
:103B500005FF050601FC01F8120900008001F001D3
:103B60007C004F004F007C00F00180010F08000036
:103B7000FF01FF01110111011F01FE01E011090008
:103B8000007C00FE0083010101010101018301822B
:103B900011090000FF01FF01010101010101830181
:103BA000FE007C10080000FF01FF0111011101114E
:103BB00001110111010F080000FF01FF01110011A7
:103BC000001100110001120900007C00FE008301B9
:103BD000010121012101E301E20112090000FF01BD
:103BE000FF011000100010001000FF01FF010A0586
:103BF00000000101FF01FF0101010B0600010001AE
:103C000001010101FF01FF10080000FF01FF013861
:103C1000006C00C6008301010110080000FF01FFD5
:103C20000100010001000100010001160B0000FF6E
:103C300001FF010F003C00F000F0003C000F00FF0E
:103C400001FF0112090000FF01FF010F001C0070BD
:103C500000E001FF01FF01130A00007C00FE008369
:103C6000010101010101018301FE007C0F08000038
:103C7000FF01FF012100210021003F001E140A0066
:103C8000007C00FE0083010101010101038307FEA6
:103C9000047C0412090000FF01FF012100210071D2
:103CA00000DF008E010001110900008E009F01114C
:103CB00001110111011101F301E2110900000100DC
:103CC00001000100FF01FF010100010001110900D5
:103CD000007F00FF008001000100018001FF007FE4
:103CE0001109000007001F007800E001E0017800E2
:103CF0001F0007190D00000F007F00F001E0017C9C
:103D0000001F001F007C00E001F0017F000F12097E
:103D100000008301C7016C00380038006C00C70147
:103D2000830111090000010007001E00F801F801DD
:103D30001E00070001120900008101C1016101316B
:103D40000119010D010701030100070008000A0124
:103D500000181110133831303378717073C8C1C036
:103D6000C38881808384848782C5C4C7C275747701
:103D70007235343732151417120207020802010097
:103D800003010903040204020503050006466972E3
:103D90006D776172652025735F25735F56330D0A59
:103DA00000436F6D6D616E64202020204465736355
:103DB00072697074696F6E257300252D3130732020
:103DC00025732573000D0A5479706520273C636FB5
:103DD0006D6D616E642D6E616D653E203F272066BE
:103DE0006F7220706172616D730D0A005570746995
:103DF0006D65202575730D0A003F0025730D0A0DB2
:103E00000A00564F5941474552203E3E2000256347
:103E10000048656C70004E6F20706172616D7300B8
:103E20004B6579207072657373003C6B6579313E28
:103E3000203C6B6579323E202E2E2E0044756D702D
:103E4000206D656D6F7279006C004C6F6164206D40
:103E5000656D6F7279007400546F67676C652064DC
:103E60006973706C6179206F757470757420746FEC
:103E700020636F6E736F6C6500000000008001505E
:103E80000080025000800350FC3F0150FC3F025074
:103E9000FC3F035025735479706520273F27206627
:103EA0006F722061206C697374206F662061766187
:103EB000696C61626C6520636F6D6D616E64732502
:103EC0007300A132C205557520C5F00E3EEB5501B9
:103ED0000EDC322B101713439CC7042B0104561120
:103EE0006A1956490A20C06A11C883C80C4EB939EC
:103EF000B70C5605AED3CD364051501711899D50A1
:103F000062CC55021B555532D0941D4D5573072573
:103F10004D1A6F9E0978490C4CFB80C030713C559E
:103F20005D05212053232E85101EEC1C1025440B0B
:103F3000B03C8300E41101C664A401422440C40BD8
:103F40005055958014510154048E269A3222A29D18
:103F5000888C62AC0771C45550C40210820881304D
:103F60003363341C0E4EB3A4200331318D8D0C4CC1
:103F700050C700880A7FE23B5474774C996E5F2FDC
:103F80000CDF530448280A810C65B90F00000000BB
:103F9000000000000000208000C06CC3C8100200B8
:103FA00000C80022218C84080B81884088409760DB
:103FB0001F13B361FB700BECC0320F7FBC0F5114A9
:103FC0000511458484B8BBAAABBB008022303323E3
:103FD000227389BB84B4BB999999457754B5B75579
:103FE0005555DB2590DC3E333221404040CE9808C9
:103FF000029244002000CC8012E034139200361567
:1040000083AFFC101C303028DE4438647D1374C646
:10401000374088403EF603122204045000FB0CC8CF
:104020008CCC4021C03AA1A7201364754E59647D01
:104030007F72D8C932E24A3B0088030100745C28D1
:10404000E2548D743B143C1141324074F3E23E1251
:1040500083D2C94009CC44C25C0E08D8FDDD335D73
:104060007C13163963CA6704110002212211510220
:1040700022C1408C84423B6BFC34FD642881F5A551
:1040800085001E8CCECFCC221C23A0C4C8A2AC209D
:10409000FC4CCCAECB328B0CCE374F44C8C523FF83
:1040A0008E3FE13C23C1E8B4E0BC23F01F4F214820
:1040B00028D6D8E0C8C808CBBA40424C80EC8B0C5C
:1040C0008DC032428AC800C32C33CA5020874014A6
:1040D000121E737117611CD5015B853FF40D3E45BF
:1040E000394B018333013E1308A54C2228358F1F1D
:1040F00002F0D8D827CB28C388030B13F5333C2C08
:104100002F0EC520484D43C1791483C58244D390F6
:1041100080038933958040D4400022DEA733040811
:10412000021B964FC5E04C1582113510BBD34C19BC
:10413000658453255D5D56544D14404053544B00E7
:10414000C1C401848C20CFC401C48C155F244C8A67
:1041500030CFC4F40068233C08E0D91D540140E28C
:10416000C86114111340D113D30DC8014C723C2FF8
:10417000CEA7E485DAA94F92F030B230A2333332C1
:10418000C333C302CC0BD80CA04C124F15550808F2
:1041900014E8C8DBEB7A8721B4CCF4804A0DEAB589
:1041A000F2D43DC41352FF04205998936EFAE240B2
:1041B000DA8A4930380CC3F0183322238C1A245F72
:1041C00055150000032300120311710008843C03FD
:1041D000CC4808007783DA00301300002C2021013E
:1041E000306088EC0C041011812448C24B8C000212
:1041F000C4300980C404F0C83832322021808ABB20
:1042000032322A44B8E2A00E82326121FB402633CA
:10421000618D204853D1208C1510234228C41812D8
:10422000FA00082500019248408000C78404140267
:104230000204048803100002082000824888400C11
:10424000090121080058E5C110FFD27520D1137271
:10425000700E8094A2FC3D3048C0D280C4F4832C00
:1042600082A832B1110641F4A1636C72890C21233A
:10427000491000A1109022F9E41F25CD0317828276
:10428000C3CCEF03C440200081A518306D83DD3B13
:10429000CD5060C4A02830C03CE05042853D0F3670
:1042A00076FFCF33ECCCCC08030310CC001EDAF140
:1042B000B0032CC2F212832CCB31C034C36058F946
:1042C000BE26C3888F2309400808314800C92058FA
:1042D0000515FDC4BF20157F505401C41853FC9030
:1042E00018608145BD430B02110208082108084CE3
:1042F00010030E08017D3E1636F1344144639311DC
:10430000D3B443A4328004AE38BF47B807FF378E1A
:104310008B2C71C7D9B80F1423EF43324BC37B13D7
:1043200044AC8F828BE201C82FF4D47E006013402E
:10433000300E7814416FB7208AC7389B840420213F
:104340003676B1330080618B843B44817B7550B2FB
:10435000C46D025008800C03648816638295D544AE
:1043600042213503A4041D6014072029D0D90A80F6
:10437000120312EE2F548AC2009084A60C50AC9205
:104380008401A7D4C8317E8058903DC81074ADBB5D
:1043900057CA33FC9CD68488331D4104220FF31284
:1043A000321193120F648ECF14C084840371C871CC
:1043B0007CCF0B33D77333B8CA7AEB0633C40FAA5A
:1043C0009501228403CB443230A38BC2A24F8C8050
:1043D000000EB0359380408E4C001601C18D609860
:1043E000408E08862806D0444C047A2023223010C0
:1043F000082321C784C48EA1C4EC311DF1004C52A6
:10440000C20087C0078000F18F17C048902C04D5E8
:10441000403220D54020720C40C354040133F94B84
:104420003338E2CC382D55F68010428D33F60082B9
:104430009404F0CE0908450432B68C8CA58C245522
:10444000C80856C84852C80856002523419532224C
:104450005632825429236B1532A204C450100544ED
:104460005115115549C5A878491055111551505687
:1044700054155155D151455785542E101714270402
:10448000030080088040E0E7921BFFFF375D8C2926
:1044900003C8B774C2503C8109A036A0C2C800212D
:1044A00008F479128273778B4058AED462A03E90A4
:1044B00040C183744408019190018F730C49558F5A
:1044C0003F03CF4E7038EEFF710CC50C6E0484A50F
:1044D0000200CAD4017E0304C002244E203C0630F0
:1044E00018E065006660E0C54E1CE020DB4E5C26EF
:1044F00050E0A2DA357D13F800DB6B710C650066C5
:104500008784C50C910C040444846500307566638F
:1045100030176673301266B15E3014665B2666B77C
:1045200088910CC55C8CEF1348F073146381004BC9
:1045300060001CC3367C14EDABDC72DC101EF81E70
:10454000E8BB31B5E47AF3E90EE960BD4CF0E8AEC2
:104550001144F0D41B0404448404446E6D2C6E0C8E
:10456000EF048C012329080D085C06A14E4E203073
:104570005ABC70E0E0DC50D4F34CA0EEE00D084DE6
:10458000320023DF3C7B1E1F00DD3F9C10069C0297
:104590005C8CFF9CA2E61C10762127A9266666D4B7
:1045A000A3FD089C3002667743A6E6A6F9083BCC3B
:1045B0004F14F714E7541BCCE766CC3F14B1071433
:1045C000135C66666666CC3FD42F14F7E108666616
:1045D000666666666666CC47563794235C514E66BF
:1045E00066CC9F54BF540B562B3010C6BB66E63BBF
:1045F0001C629CC3065CB366CC2754250366CC932F
:10460000FD089C425B5C83560FD43F945F945BA093
:104610009CA2A260739C2B5C444C47E616B6DCD48B
:10462000EB86A64454F12BB122E64816A14E30A6E3
:104630009B30059C022746466646463B6666666694
:10464000D4AF14B754A70C5FCC5BE61676768648D9
:104650005C43CCBB5C131CE508C43106FD089CD34D
:10466000FD08C8DBCCBFD4CFFD08C823FD086666B3
:104670005C7D06FD081CDBCC312FD43F8C4D1F54D4
:1046800041535C010ACC3D1FD43D0BCBCC37F846DF
:10469000E8D4311FE91ECC77D4F92B53CC3FD41F7B
:1046A00063CC0FD4E7F3CCD7D477BBA6CCE7D4E761
:1046B0007B30A7850614DFCCC7D42F2366666666D9
:1046C0006666666666CC2FD41F5C131CE50865061B
:1046D0006666E108DC49066666E1089C3D06CC9FFB
:1046E000D4EF94BFD3D4BF9487D45D0714E714D715
:1046F000CCEF5BD4479407143F14CF546FCCAFE991
:1047000006CCB7D4AFFD081CA3C49CA27D07305FC4
:104710005C8506303FDB66666666CC1366810630D4
:104720009F7BCC192FD4652FFD081C4506CC27C8CC
:10473000D43B9C1BDCC444C4A14E5C44E616864BAF
:10474000DCE90876E044844484C4C4E0B0EE8C60C4
:1047500084049C981CE2330862E21388A0069CA2A1
:10476000CE660CEF56AF301006B326061F6606E97C
:1047700008F613DC050C1E56D7EB668666468F08D6
:1047800066E908050C8CA7F623A08676A69CEAEAC3
:10479000EA43FE1FFA538E26F3FBE676A63030C6B8
:1047A000FB46C6C6FB46C65C13A2A6E77EA066D43F
:1047B0006062BBBB7EA646EF600684E0B05E5CD460
:1047C000A6F3E00E0A5A137E0ABEBAFE930CBB266D
:1047D000F64B76F62FB00E1E5B36A6CEA6061E1A38
:1047E00060AA06A0E026D49B133373C38382C272EF
:1047F0003212103070C08087C7773717113171C1FE
:104800008184C4743414183878C88884C575351503
:104810008D40A86BD14C53AE4E70382B8D405D400F
:10482000AEE04E5C6650293A8CA0BEBEBEE0C940E8
:104830002D409D4C4140C9400E882BC940B0AED19F
:104840004C213878B5407140F938A140D14CF82955
:1048500038DD4035409D4C8D4C8C60BD4CAE28C938
:10486000404540F9387D4CD1402D409D4C11445D70
:104870004038E03051A6A64E70F866A030049C582F
:10488000300B991CC4C4A0706E1C5090D0814E0E89
:104890005C62E0765A5CD0D0FC30F65A56E060A0FC
:1048A0009D0CCC606000C8CCF73004C8CC66EBE04F
:1048B0000000BC88E4E8D8787CA8FCF844404CF4BC
:1048C00074000B31B132A434D732BC168D34C436E7
:1048D000892388248A25A711AD123B13C4144315DC
:1048E0009326FA319633C934CC3543168026CF3619
:1048F0008223832484255411AB12AF13A914051508
:104900008F26BF009001AC02A203992392337F3619
:10491000EC07EE08F10979406A30642071107E4995
:10492000D6487C008F01AB0297039E041B051A0634
:10493000DF44E044EA16764067306D205E10FE49A1
:10494000FA48CA0A0ACAEAEA4A8C330E060E46E058
:104950004ACAEAEFE00050404E30C12012107F49B1
:104960001248019366930294329400954595034949
:104970008136B0FA13FE2388C85E9D38D140C14C01
:104980000ED5405D3C690CAEB05E593CFAEF0EDBD3
:10499000CC1FC8E0C4E08D40AE88FE13485E5D4089
:1049A000FAA00EE33910E32E0E7AFE4B48CC33CC3E
:1049B00023C488445CA606E641174687CECE235C16
:1049C00062EE4F4C078D180EA6AEAB4C653F213CF6
:1049D00039106ECE5C5A5E26E6433ED454D3EEC107
:1049E00016D84E3ECE6BAED8221ED8AEAEBEEB1E53
:1049F0002EAE8ECE93D83ED86EEED454B3EEB13CEC
:104A00006ED8469CEE6514EE132E62F38E42FA03C6
:104A1000DC9B4CCBD140F540A140FD40F9381E5DF8
:104A20003CB05E5846353CA606E631164116DC66BB
:104A300054EB5E9D38CC3BBEBE711829408C2B7167
:104A40001829404C776666009D3C8C3F4E5C665052
:104A500029384C13BECC604484991A4E6E5E546F54
:104A600094E7D41F5447145F9CD09CE0DC909010D6
:104A7000905090105030165CE09094F36B1CDD1455
:104A80009C505C109CE05CDD149C50DCE05CDD1410
:104A90005CE01CDD141CE0C8488D40AE0E2EBAFE52
:104AA00043884C1BCC13485EEE4CC91B8C2BAE0EBE
:104AB000CECE4E5C1050EE66F62F661B268EEE585C
:104AC000EEEEEECEEEF69F8EFB2EEE66DB4EEE9811
:104AD000EE4C1B8ECEEE8E5B2EEE98EE4C0BE6F778
:104AE000EEEBCC47C84C1F48734463C44CC38C1BCB
:104AF000842B881B8D184B6E8E0039103B26F627B1
:104B00008EB32E66009D384C5F98EE6600613C7156
:104B1000183138D8AE0E263B6EEE3BD454B726E3A0
:104B20006E4EEE6514EE133E8EF32ED4CEEE549BF5
:104B3000D88E8E4E5C50D89C90905B8A8ABEEB1EBD
:104B4000D8AE4E2ED88E1E62ABAEFAAEFA237E667B
:104B50001E8E9B98CC67CC53213C3BB05846353CCD
:104B60005D40ED38CC1B690C11448C1BBE00690CF8
:104B70000B5ED8AE98AECC1FCC1F866EDAC3D89928
:104B80003C4C7BD140E1403138F5405D3CCC6F215D
:104B90003C4CA0BEE04E5C7A360E8E4CA0234ED824
:104BA0008D18EECEE05C4ED01050D050105090D00A
:104BB000D050D0505CE0F8448460FEFE2BFE1748D5
:104BC00088B0A0E030E5A6255060E6B356069F4DBC
:104BD0004E2D2C8C63B8E64B66A646A830FDA91C6A
:104BE0008932EE4E70DCD010901010D01010684E4C
:104BF0005C1010D010D01090A8EE30E00835508C2A
:104C0000337D2CA95CBBE6E784EEBBE94CB30D0811
:104C1000355008E653F12C8C1F8884A95C8BB806AC
:104C2000F8A6E8A3EEED2C7D2C065670389C1A1ED3
:104C3000A6EEEE6E762BDCDCEEEE76DB5636DCAAEC
:104C4000AA6E2AAEF025501C6A27352C7B869C0A5A
:104C5000AE7CEE66AB2550D8F8E60122761C1BDC54
:104C6000DC76EB5670EE38AEEAEA8E8ED86E1C6AB1
:104C700093AAD8AE70AE383CAE9C6A2670AEF0A651
:104C8000986BAE70B6567F4EF02550F12C3550F132
:104C90002C352C5902EE930C1720608C604C1F5D54
:104CA0004004881A1EBA4EE0A630DFA656602E1CBD
:104CB0006A6AA070EEF0EECB314498D44AFA1BE653
:104CC000FEE00D083550512C1EBED05CA2E66321DB
:104CD0002C8C23E1202B88E12084068C95030D5435
:104CE000910CE0212C0C811C0ED8AE8C75038C89A4
:104CF0001F0D08A64E3089BC70A66056064E701C6B
:104D000030FA621F061730A80637624330B0C61665
:104D10001C10AA8C812B58EABC3006461C101006C9
:104D2000BC709806B0A0E0E68C7D3A5CD0D06B6297
:104D30001F02D3E61C4662A21B88A29076678C55A0
:104D4000021C109090505CA12636763F8C835C90BC
:104D500090533676E1238C3B5CD090492AC88C7BFB
:104D6000A0DD4CD91C0EFEB7E6734EDC905050A669
:104D700046171A952A60EEEE5EAEFCAE9B88465E44
:104D80007C464BFCA6462BFCA6464F06F12A86091C
:104D90005435508444CCC92B6E0C470C3708412C39
:104DA0000922B8FE239C514E7D2C0E76B8EEEEBE45
:104DB000EE66AEE8B8A6AEA875021C02FD263676F1
:104DC000DFA202E2578C239C10EBA61C5013024278
:104DD00013A28C239C101B8928702B367647A202C5
:104DE000E2878C4B9C501C1090D0552AA61C90DD5D
:104DF00026024213A28C2B9C5021268928A6B0A201
:104E0000AE3CE855023676FF8C635C105065222973
:104E100040DD4C8B488C3B6262B7B9281B0D2829BA
:104E200040EE703839023676478C53BEF336769FA3
:104E30008C2B9CD09126A61C105859028928B03C76
:104E4000C536A06262608CAB9C901C10D0D0A126AD
:104E50003676CF8C635C10102D26DD4CB0F08926A1
:104E60008C3B6262B7B9281B0D289B3676078C1BDA
:104E7000BE23486BB616F6E7F623A2F6BF1926A2A4
:104E80008B901CB616F6F6F6F62F8CA7C2A28C2FC6
:104E9000C23000B6D6D6A7D62FD6DF8C235C5013EF
:104EA0008C23B9281B0D28593C238C535C10101CF3
:104EB00010105C552A8C23B928930D287B8C235C19
:104EC000D06B8C23B9281B0D28BE0019401144D487
:104ED00085321C514E8C235C90438C23B9281B0DCA
:104EE000282138534E70F8BC62AEE07A6730FD631B
:104EF000DD4C5ED91C1A66F657E6F74E5C901A63D5
:104F000048FAAEBCA68646581C90A2A6464C139002
:104F100060462550E62B56064D4EA670EE38AEB0D4
:104F2000A0E0EA26BC30061C426BA2BC1C10B61BDB
:104F30009013D09090C3FC5A7A7C5CE227D05C132B
:104F40009CB67F10B64FB64F3066663B5023901329
:104F5000D00310F31CD0D01630A006CFC6E676548E
:104F60001B5C23FC9CD08C1F501390EAAA1C224B84
:104F7000D01CAAE0E65CD0A362A6DC50BEA34683A8
:104F800084A04E3004060B3007603AA0C6E34660AA
:104F90003A3A9C421F467A1ABA5A463CEEEEB6A6F8
:104FA0002550E6231C4A235C514EEA273656CB8C0B
:104FB0003D2335500C3F0C2FB85EA84EA6E8813239
:104FC0008C278801228459020C1F08DB04CB8C95A6
:104FD00003B05E7E0E0D54910C45364E7E7EEE255E
:104FE000500EE69B30F41C0A7362A22F30EBCA2BE2
:104FF0004AAAEE3EEEFBAE512C0A4E9C90D0AEA0DB
:105000005ACE1C50FE5C50D01CD0D090D0D0602B1B
:105010009C509C424E1CD0B656FCA6BC430C1F0CA8
:10502000AB255006F8661F4663601CE65316D01683
:105030004BB636DCF0E030FCDB661C50BB25500E76
:1050400030F0E666952AAE9D2CE035500656703855
:10505000B6B660CECEE3AED8AE5E5A0EE6EB9C504E
:1050600062D0BAA05A76F3DCD060269CA0DA6062E7
:10507000E31C223FA05C5050905A605CAAE076F698
:105080005F1CD02AA630FDA66A1746F0E02623351D
:1050900050E625505EA84EE6E8E0B0BE0E4E5CD06D
:1050A0001940FE1BFD40D91CFE134EE04EBE2626C5
:1050B000D84EDC5050905CE016CAA78D4FB7A6D0F2
:1050C000A14CC84801504C378C33350CBB8C605E0A
:1050D000AD44D1404CA3B14CF5402940CC47810CA4
:1050E0000EB01EAEE0A140D140213CE940CC1F8172
:1050F0000EB14C6B350C1140D140B0350C1940ED60
:10510000385D3CE940694E01508C600E5CA24A2F2C
:105110004E7A366B0E19401ED140B05E350C1540EC
:10512000E140693C694C713201508C609D38D1403E
:10513000F5405D3CF540E140693CB05E2140694C82
:105140009B6556F6332627DAFAE7BA2550BAAB65DF
:1051500046882D56390C390C390C7BB928F0AE53E2
:10516000DD4CF0F0B023DD4C4E68B8E61F30FE9900
:105170001C5902091C4E702868A87030E69329401B
:105180007118EE3A46232940F83902690CE34E992A
:1051900002B05D40DB3550E6672550440CA70C9FFC
:1051A0002D2C84BBCC3381008C170B6E212C6EBD53
:1051B000220484E94CE667EED704750235500C579B
:1051C0000CCF0884E609231D1E7D2C846B842908DE
:1051D000E00D54461C1066FB811C590248A0DD4CB2
:1051E000D91CD84E70D828E6F62B9A26E3FA46BE8C
:1051F000BA0E66689C0A254CD91CD84E70D8A829CE
:105200004CFA1F4E224C17BEAE381940280E78BEFD
:105210001E1940AEDD4CAE684E70B80E384C279368
:10522000550C1540BE77FE6F23550C4EEE3B435593
:105230000C1540FE7D2C5502550C4EEEC7CB355259
:1052400088091CC14CB0280ED14CF84C1778990C29
:105250000D40C14C389D38D14C384C17B8990C01D1
:1052600040C14C4C1F48030EB02138990CD14C78EA
:1052700001400E62990CD14C0D40BD4CB0E8AE9986
:1052800002091C490CF8AEFA271C514E593C394012
:10529000490C78AE593C3902091C44D14C2EFAAE67
:1052A000FD40D1404C27A9401B45408D4C35409DC9
:1052B0004C7D4C4C27284823394038DB091CE50E2F
:1052C000091CB10C93091CD14C78EEF84140EE3B1F
:1052D0000CCF48BB8CDF4806B0551C1C6263EADC6F
:1052E000E3E68C1F449B0C8783A214FFD4274C1742
:1052F0007ED4D48EAAEE3CDCCABCAEEE5C1EA05AB4
:10530000870EAE6E4B8C1B0C9FFA6502BE44F0DB21
:10531000428FA6FAE326935CEA8EB0A09C1D4086DD
:10532000061CD62B8A838A06AEFCAE261C5E2FA6F0
:10533000EE8ADBA66E11445439029B9CA2A2A2D332
:1053400084488CD7611C442E5C22029CD84670F89D
:10535000AAA6E8A6AAD86A085A0F046AF3FA13EEB6
:10536000DCD0EE3EB30CA72E1B0E03C94AAD46ADF2
:105370004A0E514884B02938094E0EBE77E1407B71
:105380003540638D402B550C66662E7A58463E5E3E
:10539000D8065E139E0ED8DCDC8E132E62F354CB3F
:1053A00098AE5898FE1B66CEAE5C4ABFEEAE5C0E61
:1053B000E66B3A5BC62622DE6EFA604E1EE0C6C37E
:1053C0006E63424F66EAE32EFAAE4ED84E5C50EE64
:1053D000AED8AE4BFA4B8D402E7A58463EFAEBD8FB
:1053E000465E139ED85EAE6E2E2BD8EE66D85C4E0F
:1053F00013228EF32EEED4D4D3AE98A93AAD484EF4
:10540000585148EEC3550CA10C1940386666005B34
:10541000BE008D4019422EFAAE5E239C514E3ECE08
:10542000EEB13A6EEEEE0EEE5A0EEEE613BA4E9C6A
:105430004217AE8E4E6EDC50CE4B22CEF34EEE9423
:105440000FD4CAC3C848D1186916C848C8D118951E
:1054500012D1185516D118C1120E7118EEB0293894
:10546000AD00613E0EAD0021387118693E88FAA08A
:105470000E8E2626065C4647D4941BCEE066D34E9D
:10548000DA8C93DCD42309102BDC0910D4D4091056
:105490000ECE7D3A0E0110DCD417DC0110EE4EEE7C
:1054A000938831448C9D3A98D44AB13A5EE05E3399
:1054B000DC101BDC501EF8FCD88404D83C601EE8CD
:1054C000590221401B19401144F05CE0B04C60537C
:1054D00011440E4C27B05D40AE584E7078A84E7007
:1054E00038689828E0EE4E70380E7828B868D3BE39
:1054F0000021401BA9404E7078A83868CEBE1E28F7
:10550000F8BA9CEAEAEABAE8AA8A8A8AE071404EC6
:1055100070EED8F81A9ABABABA1CEAE6E838EE7809
:1055200028B868BA463CFED8EEE04E7038BE5CEA59
:1055300028F89CEAEAEAAAA6E8834E70389C534E03
:1055400070781C2B4E70B89CEED8F8D4CE14EBFEBD
:10555000AED8E0D14CF8E138D140490C38D3D14C29
:1055600078AEF8E538D140D14CAE7863D14C78E1D3
:1055700038D140D14CAEB8213835408BE140EB4EAC
:105580001B4EBE5C502BAEBE2E7A58463E5ED81CDB
:10559000D4763654E3EEEE6BD86EEE4B2687D86E9B
:1055A00026DFAED80E23D8AE2BD8AED86E9E5E5B6B
:1055B0008E1E263BD8FCD86EA66E264B66CEBE1E2F
:1055C000D4D4C34EAE98EE2E767676007D3A2EFA7F
:1055D000AEDCCED86ECEF66026E63B66EE1ED44E2E
:1055E000CF66E0A643653EFEEFF6DF0E8E1CEE8A28
:1055F0005C4A8F66061B36E04E22CE3EEEC21BAAE8
:10560000260EC223EE2EFBDE338A6E262EFB6A6246
:105610006B7E5BEE865A5E2A4EBAE04E1C985CD4D6
:1056200076F3CEEEB00ED6875653DCD42766E3432E
:105630004E4BD41437A6E38A3A5B1E7E06A6166646
:10564000D3268ED40AA3FA174EA05CF62B86F61F3B
:1056500086E0F61F4E2B4A6A56D4D4E0BE6E8E58B2
:105660008E4E27980EE026CB5C626E993E2EFAAEE7
:1056700084045E13081E1A6ECEE673CE5E7FDCD401
:1056800094214B26DB8D48C351485C336E66AE33A4
:105690003A8EF32EEE66539CE22B62E24F225C437D
:1056A000AEFAAEE26B4E5C6A0E1C500C13A66E0E88
:1056B0004C3BD140FD40A1408C1BBE1EF93A228ECE
:1056C000F32E5447EE66D4EE0D46EE4C2BBD48AE9D
:1056D0006EDC909CFA83DCE22B628E587B268E7EF9
:1056E000A3463C626E0E0C213D3BAE7EF32E7E98AF
:1056F0003B588EEEEEEE0E6ECEEE2798AEE066CB09
:105700008ED826893E6E5A5E0E0C1B69444C1BD106
:1057100040F540D946EE5C90D0109050105010509B
:10572000905050100B4E54977A103AD4DF543714DF
:105730007F94BF54E79CD05C6B9050D05010D050F9
:10574000101050905CEEE0D0501050D0501010105F
:10575000D0D09C931CD0D0101050D03068DC3B5C73
:10576000D0D0D01010D0505CEB5CD0D030311CB316
:1057700030339C932EFAAED14084C14C0EB05EBB48
:1057800006BAF633653EE6EB66EE5ADFE64FBE1E1E
:10579000FEFE1EFE1388C14C5E6D488D422EFAAE91
:1057A00048DA7F3540FAF398FEDF2EF93A2EFAAE4A
:1057B00044043E5E87DA73A606E67B461BA6080E07
:1057C0005E5A5C8A62228E588B5CCE62AE4EE94E87
:1057D000422766EEE3D8993C8BF540B344043EAED5
:1057E0000E26E6B35E57AE6D445C4EA60E6E3B08C9
:1057F000CB54F7D43E26DB7B8E7EF3982EBE3B3E09
:105800006EEED4949BAE8EEAEAEAAE9CD086C6E3F6
:105810005C8EEE8D48414CFAE3D4BB2E9C822E8EDA
:105820004D480C376E8E6E2E6E1C414CFA3B8EDB53
:10583000EEDB8E235EEF665E0C1BBE009D384CCB0C
:105840003540313898FEBD46A6EEDB8EBD486E5C15
:105850001B2E62F34226DCE08CA04ED85148EE6944
:105860003E5E475D3ED14C5846FA1D36693EF540D6
:10587000E30E4E7038E030E0DB30FDC3B80EF8CEFA
:10588000BECECE761356E8AEA8AEE066665C422782
:10589000FAA6E3AEE01C4E0404C4606E2ED436D4E7
:1058A000EB1C9090901090BCAE1C1D544C29038CA6
:1058B0002F0C60910C4E70606E28F83051A6E86095
:1058C0000000EE4BF643A6300586061388B0E0F6DE
:1058D000FFD91C0EB0CEFE2F4E8F95464E375C4A38
:1058E0002236E0E65B66E6434EE0E62366E6876145
:1058F0002C0EB01940F540D140ED384E509026297D
:1059000038D1404E5C2650502140A92C1050353CD7
:105910004E26D010D010102140E940A92C50D0358F
:105920003C4E269050D05050BD40F5404E5CD029A2
:1059300038DD404EBED84E101010353C4E1066215A
:1059400041E940B14C4E66D84E50501050D01050E6
:10595000D0D09010D02940F540A10C2940A140F5AD
:10596000404EBE665C50BD400940B948F938DD4044
:10597000B944D140612C2EFA0ED140DA5BB02140FF
:10598000B14CA140FD409BF540F93A30FEC54E3088
:10599000FFE38C3132600CD7DC501C62335427DCBF
:1059A0007ED34C3B7E37A2D4442BBE025437B0C5C5
:1059B0003A069C4A4704C14CF80A65025C4A279C97
:1059C00002138A5D3AFE2F31444EA0653E811C0DC4
:1059D00054C14C0D54B0550C1C428F1540FE6F68DD
:1059E0000EB0288C4F1540FE2B7828B068C14C5C57
:1059F000EE1F50334E50280E781940D14078BD4CE0
:105A00006EA32E7AF540680EB819408C2778613C59
:105A1000F938F6373BE140F9388D422940A025504E
:105A2000FA5C5050D010D05090909050237AFA7A6F
:105A3000DC133A62F354BB19483AB8BAA8BA4E66B6
:105A40009D39390260E61686662550E6952A58F893
:105A5000E61F30FC0698DCD01C6A1F883C3EFEA680
:105A6000065670381E7EB6561B3CDB6A6A8B3C7E3F
:105A70003EDF668C334CB74884CB1676A6C3BEBCDB
:105A8000F6668444E05CC44813448460795C4E70DC
:105A9000E0AE28FE1BFE4F0C3B9CE21FD013D0A8AB
:105AA0003C364F450CD61B5C903C4EB83C365F45AF
:105AB0000CD61B9C107CEEEE4EB83C364F450CD6F7
:105AC0001B1C103C4EB87C364F450CD61B9C10FC62
:105AD0004EB8BC3657450CD61390FCEEEE4EAE7564
:105AE0005C0EB87C365F450CD61B5C90BCEEEE4E6F
:105AF000B8BC364F450CD61B5C90BC4EB83C365FEC
:105B0000450CD61B9C103CEEEE4EB87C365F450C27
:105B1000D61B5C107CEEEE4EB8FC364F450CD61B07
:105B20009C10FC4EAE615C8C234C3D5FF8FE434EF6
:105B30003008A8300C3B4E300CA8300868A0381E46
:105B40007E877E577E73B8BCEEEE4E7C1B787C4E13
:105B50006E815AA0BE600EFC9C02788C234C174EBE
:105B6000A297A20FA25FA27FA2F7A25FA27FA2F7D5
:105B7000A2477B7C4EB87CEEEE4E6EB87CEEEE4ECD
:105B8000B8BC4EC37C4EB8BCEEEE4E6EB83C4E6315
:105B90007CEEEE4E6EB87C4EB8BC4E9CB0FE231030
:105BA0009C427870686E6D5C8C1B4C37F85A46FED0
:105BB000FE3B1C10FE1B1C105EDC8C1350695C4EFF
:105BC0005C0C13501CCC1B223BA0D423E01C505572
:105BD0005C38EEA0E020E00E7870682B0EB870A85C
:105BE0008C2BCCA048E04C60C8CC60889D0EA01CDB
:105BF000109C50201378EE68A886910C4E5C906E35
:105C0000F7CCEB3026065ABC3006203C5666876E31
:105C1000663028060F4E9C9090683CA89D02664E08
:105C2000A02660A6E33C4B4E26263C234EE34E5C6A
:105C3000F0514E811CB02844D95C6ECD00AEF09876
:105C40006E5FA01C100626E630187CBA233A7A3321
:105C50003046DB26CB86468748D95C6EB0CE4E3ABE
:105C600030F3A66E47CD000E986E174E7038704E0A
:105C70006E68A8CCA0848102A0CD00F0F0D8D8D85E
:105C8000D8D8D8EE6ECD00CE4EB15F584E300770EA
:105C9000EE384EAE4CA72EAED8F04E38D8F030E0ED
:105CA000AEEE66A06E664B563B8E00630920F8E6AA
:105CB00037300CE8E6E6C8CC2366E3E09D0CCD4E19
:105CC00000000304050A08060BFF0209070D010C7A
:105CD00000FF2025692025692025692D25690020E0
:105CE0002025633A256900202020205F5F7C002C5E
:105CF0000044697370206F66660D0A005553455263
:105D00000046004700424547494E00524144004486
:105D10002E4D59005052474D0055534552202020DA
:105D2000006620200067202000424547494E202081
:105D30002020200052414420202000442E4D592094
:085D4000202000432020200078
:105D4800F93D000000000000610D0000113E000058
:105D5800163E0000143E0000FF000000B9060000D7
:105D6800203E00002A3E00008737000000000000A7
:105D7800A50400003C3E0000163E0000483E00001E
:105D880000000000B10500004A3E0000163E000079
:105D9800563E00000000000011070000583E0000B9
:105DA800163E00000F000000F4010000040103018A
:105DB8000201010411040F04170416011801000060
:105DC800195D0000215D0000255D0000295D0000CF
:105DD800035D0000345D00003B5D0000435D000092
:105DE800145D000000171B243E4253697505020527
:105DF8000804080B08040405010504090809040639
:105E08000807020602040206010604070103080344
:105E1800040C080D020C0203020C010C040D010D08
:105E2800080D040802080807080202070408010808
:105E380004090209010A080B020A0201080A010AF8
:105E4800040B0102080204100811021002110810C4
:105E58000110041101120212011302130812080F93
:105E6800081204130113041402140115021508146E
:105E78000817081404150115041702170119081A40
:105E88000219021602190119041A01160816041B30
:105E9800021B081A0818021A041B011B0418081808
:105EA800040B042020202020202020202000000097
:105EB80001000000FC5C0000015D0000035D0000C3
:105EC800055D0000035D00000B5D00000F5D000034
:085ED80073370000145D0000A7
:04000003000035259F
:00000001FF
